:1000000055AA55AA0200000036700000000000004A
:1000100028F2000000000000FA00000000000000CC
:100020000000000000000000FA000000105A00006C
:100030000008000000000000000000007D025B0ED0
:10004000E695515E83160000196AAEA17CE9FFFFB8
:1000500000021000E1000000B7460000A10100000E
:10006000ED010000390200008502000000000000E0
:10007000000000000000000000000000BB4600007F
:10008000C346000000000000D1020000CB46000083
:10009000D3460000E1460000E9460000F7460000B4
:1000A00005470000134700001B47000029470000D8
:1000B00077470000DF020000374700003F4700009D
:1000C000000000004F470000794700007B47000018
:1000D000894700008B4700008D47000067470000FC
:1000E0006F470000574700005F4700008F47000040
:1000F000914700009F4700004747000000000000B4
:1001000000000000000000000000000000000000EF
:1001100028F2000001000140000000000000000083
:1001200000000000000000000000000000000000CF
:1001300000F002F800F03AF80AA090E8000C8244BF
:100140008344AAF10107DA4501D100F02FF8AFF29C
:10015000090EBAE80F0013F0010F18BFFB1A43F0A5
:1001600001031847B4560000E4560000103A24BFBB
:1001700078C878C1FAD8520724BF30C830C144BF0C
:1001800004680C607047000000230024002500264E
:10019000103A28BF78C1FBD8520728BF30C148BFEA
:1001A0000B6070471FB51FBD10B510BDDFF80CD038
:1001B000FFF7F8FF04F0AFFB04F0C8FF00021000E7
:1001C00003B4FFF7F1FF03BC04F0C8FF40BA704767
:1001D000C0BA704772B6784600F10A004DF8080CB4
:1001E00062B630BF00BF704740BA7047C0BA7047B0
:1001F00011484FF00F0100F8011B4FF0010100F80A
:10020000011B4FF0020100F8011B4FF0000100F844
:10021000011B00F8011B00F8011B00F8011B00F88E
:10022000011B1EF0040F0CBFEFF30880EFF30980F1
:100230004FF0020103F0EABA0002002011484FF02B
:100240000F0100F8011B4FF0010100F8011B4FF0F6
:10025000030100F8011B4FF0000100F8011B00F83A
:10026000011B00F8011B00F8011B00F8011B1EF028
:10027000040F0CBFEFF30880EFF309804FF0030188
:1002800003F0C4BA0002002011484FF00F0100F83B
:10029000011B4FF0010100F8011B4FF0040100F8B1
:1002A000011B4FF0000100F8011B00F8011B00F8D2
:1002B000011B00F8011B00F8011B1EF0040F0CBF0E
:1002C000EFF30880EFF309804FF0040103F09EBACA
:1002D0000002002011484FF00F0100F8011B4FF001
:1002E000010100F8011B4FF0050100F8011B4FF060
:1002F000000100F8011B00F8011B00F8011B00F8C9
:10030000011B00F8011B1EF0040F0CBFEFF3088067
:10031000EFF309804FF0050103F078BA00020020E6
:1003200000B504F0E7F95DF804EB00F02FB81EF01B
:10033000040F0CBFEFF30880EFF309804FF00001CA
:1003400003F064BA0A484FF0FF0101704FF000005B
:1003500080F311884FF0000080F3098805484FF0C2
:100360000201017062B604484FF08051016070478D
:1003700022ED00E0F202100004ED00E002484FF030
:10038000805101607047000004ED00E04FF0200054
:1003900080F31188EFF3098098B112480068124980
:1003A0000968884217D0EFF309800E49096820E9EF
:1003B000F00F886000B50B48006804F080FB5DF822
:1003C00004EB084808490A68026000688168B1E8DF
:1003D000F00F81F309884EF0040E4FF0000080F317
:1003E00011887047F4021000F8021000EFF311803A
:1003F0004FF0200181F31188704700004FF000009A
:1004000080F311887047000062B6704772B670477B
:1004100010B5022000F00AFA032000F007FA0420C9
:1004200000F004FA052000F001FA062000F0FEF9C1
:10043000072000F0FBF9082000F0F8F9092000F08F
:10044000F5F90F2000F0F2F94FF00051002001F80B
:100450004A0F8871F022CA710F224A70F949086266
:1004600088620863886008618861C8604861C86103
:100470004862C86248630621022000F0F6F90621AE
:10048000032000F0F2F90621042000F0EEF9062125
:10049000052000F0EAF90621084600F0E6F90621F9
:1004A000072000F0E2F90621082000F0DEF904211F
:1004B000092000F0DAF906210F2000F0D6F9022019
:1004C00000F0C8F9032000F0C5F9042000F0C2F9DB
:1004D000052000F0BFF9062000F0BCF9072000F06D
:1004E000B9F9082000F0B6F9092000F0B3F90220AC
:1004F00000F091F9032000F08EF9042000F08BF950
:10050000052000F088F9062000F085F9072000F0AA
:1005100082F9082000F07FF9BDE81040092000F0C2
:100520007AB94FF00051C98C4FEA90100A06C549BC
:1005300001D5C54A00E0C54AB2FBF0F0086070473B
:100540004FF0005090F84A00000700D0012070479B
:100550007047BF4900200860BA498860C86070478A
:10056000B84AD160642148430A2190FBF1F0B0F50C
:10057000803F06DBA0F57F40FF3890604FF6FF70AC
:1005800002E0002180B2916000F07FB9AD4910B562
:100590008868B0F5803F06DBA0F57F40FF388860B3
:1005A0004FF6FF7003E030B10022C0B28A60BDE8B0
:1005B000104000F06AB9CA68FFF7CBFF12B1BDE87E
:1005C000104010470020FFF7C3FF10BDA0490020D6
:1005D000091D08609B49086148617047994A51614B
:1005E000642148430A2190FBF1F0B0F5803F06DB1F
:1005F000A0F57F40FF3810614FF6FF7002E0002148
:1006000080B2116100F04BB98E4910B50869B0F5A0
:10061000803F06DBA0F57F40FF3808614FF6FF7092
:1006200004E0002806DD002280B20A61BDE8104027
:1006300000F035B94A69FFF7C9FF12B1BDE81040B3
:1006400010470120FFF784FF10BD814900200831C9
:1006500008607C498861C86170477A4910B588692B
:10066000B0F5803F06DBA0F57F40FF3888614FF68C
:10067000FF7003E030B1002280B28A61BDE8104013
:1006800000F017B9CA69FFF7E0FF12B1BDE81040EA
:1006900010470220FFF75CFF10BD6D4900201031AC
:1006A00008606849086248627047664910B5086A80
:1006B000B0F5803F06D3A0F57F40FF3808624FF6C3
:1006C000FF7003E030B1002280B20A62BDE8104042
:1006D00000F0F9B84A6AFFF7E0FF12B1BDE8104038
:1006E00010470420FFF734FF10BD59490020143192
:1006F000086054498862C8627047524AD1621168E2
:1007000048430A21B0FBF1F0B0F5803F06DBA0F5CD
:100710007F40FF3890624FF6FF7002E0002180B208
:10072000916200F0DBB84FF00050B0F85A00454934
:10073000096908447047434910B5886AB0F5803F9D
:1007400006D3A0F57F40FF3888624FF6FF7003E0C4
:1007500030B1002280B28A62BDE8104000F0BEB81D
:10076000CA6AFFF7C2FF12B1BDE81040104705206A
:10077000FFF7EEFE10BD4020C10581F82100704753
:10078000334800211C3001604FF000524FF6FF71DA
:10079000A2F866100121016070472D4900201C312C
:1007A000086070474FF0005090F82110C90606D538
:1007B00010F8211F21F01001017001207047002066
:1007C000704710B504460F2000F044F80F2000F0E9
:1007D00022F81C4844604FF00050C18C090602D535
:1007E0004EF6602101E04AF6C871416518490120C2
:1007F000B8310860091D086010BD10B50F2000F069
:1008000015F84FF00050C06C0E4920F07F40496849
:10081000BDE81040084700F01F0201219140400947
:10082000800000F1E020C0F80011704700F01F02C6
:10083000012191404009800000F1E020C0F88011C2
:100840007047000000021000C0270900D0DD06003C
:100850004009002200F01F02012191404009800060
:1008600000F1E020C0F88012EAE74907090E0028ED
:1008700006DA00F00F0000F1E02080F8141DDFE739
:1008800000F1E02080F80014DAE71A4900220A603B
:100890004FF00052A2F8580001200860D0E7154937
:1008A0000022091D0A60CA06A2F85A000120086049
:1008B000C6E71049002208310A608A06A2F85C00E7
:1008C00001200860BCE70B49002210310A604FF09C
:1008D0000052A2F8600001200860B1E7054900223B
:1008E00014310A604FF00052A2F862000120086043
:1008F000A6E700004009002210B55B4C00202060F4
:100900005A4800F09BFD0120206010BD10B54FF04B
:10091000E0214FF08060C1F88001C1F880025449A5
:10092000A02081F80004FFF7E7FF4FF00051C88CCA
:10093000CA8C00F00300120600EB400001D54D4ABE
:1009400001E04C4A303A12F8203001F8983F02EBAF
:10095000800042784A7082788A70C278CA700279C0
:100960000A7142794A7182798A71C279CA71027AAE
:100970000A72427A4A72827A8A72C07AC87210BD4A
:1009800070B54FF0005400F07F00049D84F88D0096
:1009900084F88E10A4F8942001213748002283B1F6
:1009A000C0F8801194F8913023F0700384F89130EE
:1009B00094F89130702606EA05152B4384F891309F
:1009C00001E0C0F8802114F8923F23F03403237033
:1009D000C0F84422C0F84012D0F89C110129FBD184
:1009E00070BDF0B54FF00054DDE90765DDE905C7DE
:1009F00000F07F0084F88D0084F88E10A4F8942015
:100A000084F88F30A4F896C001211B48002287B1DA
:100A1000C0F8801194F8913023F0700384F891307D
:100A200094F89130702707EA05152B4384F891302C
:100A300001E0C0F8802114F8923F23F034032370C2
:100A4000237843F02003237016B1C0F8481201E068
:100A5000C0F84822C0F84422C0F84012D0F89C11D7
:100A60000129FBD1F0BD000084140022AA820600F7
:100A70001AE000E06C51000000100022374801210C
:100A800001600021016070473548012101600021AB
:100A90000160704700B54FF0E0230122C3F88021C8
:100AA00003F5C073FFF7F0FFFFF7E8FF2C480838A5
:100AB0000260A02083F88002C3F8002143F8802C54
:100AC00000BD2749083910B1002008607047012097
:100AD000FBE723480121783801600021016070475D
:100AE00010B572B61F490C78002104E01D4A521C53
:100AF000525C4254491CA142F8DB40F6FC0000F075
:100B00009DFC62B6204610BD144901201C390860C6
:100B10007047144820300078124921310978401A72
:100B200000F03F0070474FF00051027881F800223A
:100B3000427881F80122827881F80222C27881F815
:100B40000322027981F80422427981F80522827910
:100B500081F80622C07981F8070270475C84002280
:100B6000940500220004002010B50A2000F05AF875
:100B70000B2000F057F80A2000F05FF80B2000F07F
:100B80005CF805210A2000F063F805210B2000F035
:100B90005FF84FF000507F2100F8351F4170C170A1
:100BA0000021C17101724172817210BD0123834025
:100BB000D8B24FF00053002993F8361001D001430A
:100BC00000E0814383F8361013F8381F0AB101435F
:100BD00000E081431970704701238340D8B24FF081
:100BE0000053002993F83C1006D0014383F83C10D1
:100BF00093F83E10014305E0814383F83C1093F8DD
:100C00003E10814383F83E1013F83D1F22B101438B
:100C100019709978014303E08143197099788143F1
:100C20009970704700F01F02012191404009800037
:100C300000F1E020C0F88011704700F01F02012190
:100C400091404009800000F1E020C0F88012704718
:100C50004907090E002806DA00F00F0000F1E02035
:100C600080F8141D704700F1E02080F800147047F0
:100C70007047FE4BFE4A998A814203D2401AD080C7
:100C8000084601E00021D180DA68FA491047F748A8
:100C900010B500698047F649C88810B1BDE810401A
:100CA000E7E78968002903D0BDE810400120084724
:100CB00010BDEE4810B500698047ED4C4FF00000C4
:100CC000A16819B188470020A06010BDFFF7D0FFD0
:100CD00010BDE749CA780B7952005A43E34B0878B4
:100CE000D2B29B6840F48070C96818470146182248
:100CF000DE4804F031B938B5DD4A8179132311712A
:100D00004179D170027901F0070102F01F028DF8DC
:100D100000208DF80110C078032200F01F008DF82C
:100D20000200D248694644681846A04738BDF8B565
:100D30000446007CCD4DC0F34002014662F35F01E2
:100D4000C0F3800241EA8201C0F3C00241EAC2015D
:100D5000C0F3001241EA0211C0F3401241EA42110D
:100D60008DF800108109607C272300F0010241EA20
:100D70000211C0F3400041EA40108DF80100607C90
:100D8000C0F38001C0F3C00241EA0211C0F30012B7
:100D900041EA4211C0F3401241EA8211800941EA5E
:100DA000C0108DF802006E68032269461846B047ED
:100DB000E0792B23C0F38002014662F39F01C0F368
:100DC000C10241EA0211C0F3401041EA80108DF8DF
:100DD0000000607CA17CC00901F0030140EA011021
:100DE0008DF801006E68022269461846B0472D262C
:100DF0002B680122694630469847A17C9DF8000087
:100E0000C1F3800108438DF800006B680122694638
:100E100030469847F8BD10B50446FFF76CFF2046F2
:100E200000F04FF92046BDE8104080E738B53D217D
:100E30008DF800108D49044612204B680122694646
:100E40009847A088FFF715FF38BD10B5044600F09D
:100E50007AF92046BDE81040E8E7F8B5834C122542
:100E60000646236801226946284698479DF80000F7
:100E7000012240F008008DF80000636869462846AA
:100E800098474825236801226946284698479DF8D7
:100E90000000012220F0060040EA46008DF8000024
:100EA00063686946284698472368012269462846B0
:100EB00098479DF80000012240F001008DF80000E5
:100EC0006368694628469847F8BD38B5674D482499
:100ED00001222B686946204698479DF800000122B0
:100EE00020F001008DF800006B68694620469847A5
:100EF00038BD38B55D4D2A2401222B68694620464D
:100F000098479DF80000012220F0100040F00100F9
:100F10008DF800006B6869462046984738BD38B5A3
:100F2000524D2A2401222B686946204698479DF895
:100F30000000012220F001008DF800006B68694676
:100F40002046984738BDF8B5484C442506462368E6
:100F500001226946284698479DF80000012240F08A
:100F600082008DF8000063686946284698472D2561
:100F7000236801226946284698479DF8000001220F
:100F800020F0FC0040F08E008DF800006368694698
:100F90002846984714252368012269462846984721
:100FA0009DF80000012220F0070040F001008DF8BC
:100FB0000000636869462846984715252368012282
:100FC0006946284698479DF8000006F01F0120F06A
:100FD0001F0001438DF8001063680122694628460E
:100FE0009847F8BD2DE9F843204C1325174688464D
:100FF00081462368012269462846984701269DF8C4
:10100000000006FA08F120F01F0001F01F01014363
:101010008DF80010636832466946284698472725B0
:10102000236801226946284698479DF80000BE4083
:1010300020F03F0006F03F0101438DF80010636887
:1010400001226946284698472E25236801226946D1
:10105000284698479DF80000012240F00C008DF8CA
:101060000000636869462846984705E004031000BD
:10107000380210003F0C00003E2023680122694620
:1010800098479DF8000000F0300189F80010BDE895
:10109000F883554B40F480701B681847524B40F45E
:1010A00080705B68184701B506209DF8001001228A
:1010B00001F01F018DF800104B494B6869469847B5
:1010C00008BDFEB5494D0446007828706078687008
:1010D000454EA078A870312733680122694638460A
:1010E0009847E07940069DF8000002D540F02000C6
:1010F00001E020F020008DF80000E179090602D51A
:1011000040F0800001E020F080008DF8000073685E
:10111000012269463846984721893220C1F30801E7
:10112000ADF80010E168CDF8021029788DF80610AE
:1011300069788DF80710A9788DF80810736809226E
:1011400069469847FEBD70B504460168274886B0D9
:10115000254D8160A168C160E1680161217C162094
:1011600001F001018DF80010617C8DF80110A17C67
:101170008DF8021000218DF80310A18A0F22C1F30F
:101180000C01ADF80410E18AC1F30B01ADF80610B3
:10119000218BC1F30B01ADF80810618BC1F30B017A
:1011A000ADF80A10A18BC1F30B01ADF80C10A17FB3
:1011B0008DF80E106B686946984731262B6801221E
:1011C00004A9304698479DF81000E17F20F01F00E9
:1011D00001F01F0101438DF810106B68012204A972
:1011E0003046984706B070BD040310003802100066
:1011F0004FF0E0214FF48030C1F88001C1F8800247
:101200007249A02081F80004704730B5704C012568
:101210002560E50603F03F0385F86B30002304E00A
:1012200051F8235040F823505B1C9342F8DB002018
:10123000206030BD30B595B00446302103F0E8FEA3
:101240006448006800906348001D00680190614890
:101250000830006802905F480C30006803905D48D9
:101260001030006804905B481430006805905948BD
:1012700018300068069057481C30006807905548A1
:101280002030006808905348243000680990514885
:10129000283000680A904F482C3000680B904D4869
:1012A000303000680C904B48343000680D9049484D
:1012B000383000680E9047483C3000680F90454831
:1012C0004030006810904348443000681190414815
:1012D0004830006812903F483F494C306FF002059B
:1012E00000681390009888424DD1A810A061206139
:1012F0002060A062E062E061206203A8029900F031
:101300006FF8019981423ED10B9845F2AA5180B203
:10131000884208D10498C0B2A061139A92B28A425E
:1013200000D0801DE0610C9880B2884217D10398EC
:10133000039A00F47F40D2B240EA0240039AC2F31B
:1013400007421043254A904203D30598C0F3012079
:1013500000E000202061059800F00F0020600D984B
:1013600080B2884201D10698A0620E9880B288426D
:1013700001D10798E0620F9880B2884201D10898A5
:10138000206215B030BDA56125612560A562E562CA
:10139000E5612562F5E710B50446142103F038FE37
:1013A0000C487C38006820600A488038006860601B
:1013B000084878380068A060064874380068E06023
:1013C000044870380068206110BD000010E000E0A3
:1013D000441B0022B41E04005C000D6000010200EA
:1013E000F0B5074600200346184E10E057F823508A
:1013F00003224FEAC20C45FA0CF484EA2064E4B2FA
:10140000521E56F8244084EA0020F2D55B1C8B4221
:10141000ECDBF0BD70B5054600200C4C0246103CDC
:1014200009E0AB5C521C03F00F0604EB1313A65D3E
:101430001B78304418448A42F3DB70BD08B5009035
:10144000401E00900028FBDC08BD0000AC510000ED
:101450004FF00051C88C4C4A00F0030012687AB17A
:1014600001280AD0022806D0032802D04FF41670B3
:101470000EE046200CE096200AE04FF4967007E05C
:1014800001280ED002280AD0032806D04FF4E170BC
:10149000401E21F8520F088070473220F8E76E2076
:1014A000F6E7DC20F4E748F61971480720F82A1F10
:1014B0000B2180F83E1000214183022180F8C010EA
:1014C0004FF008510120C1F8D4032F499839086022
:1014D0002E49086070474FF0005141F29840C8848F
:1014E000B6E74FF0005140F29A70C884B0E74FF071
:1014F0000050C08CA0F5A051983901D00020704751
:10150000012070474FF000518A8C60F304028A84F6
:1015100070471F48016841F00401016070471C4892
:10152000016821F00401016070474FF0005108810B
:101530007047174928310968016015491831096851
:10154000416013491C3109688160114920310968E3
:10155000C1600F492C31096801610D490C390968D6
:1015600041610B4914310968816170474FF00050A7
:10157000808870474FF00050807970474FF00051DD
:101580004C2081F820007047DC040022EC1B002274
:1015900010ED00E030B41DC8474981E81D0001216D
:1015A00030BC002003F0BCBA2DE9F84F43480124B9
:1015B000006810F86C5F417890F846004D4300F0E9
:1015C000030004FA00FA3C486421103003F020FDC7
:1015D0003B4802F049FE3A483A490471097809B992
:1015E00002210171DFF8D080002408F1100B37E0F0
:1015F000DFF8CC90032734490026C9F8001048468C
:1016000002F036FE00226B460121104603F0D8FAA4
:101610000121002003F0B3FA98F8000068B102F04D
:1016200028F97F1E002F0BD0E9DC002E2ED04FF0C2
:1016300000005946D8F804200FE04FF00106F4E707
:101640004FF0040002F009FEEFE751F8203032F9C4
:1016500010703B4441F82030401CA842F5DB641C6C
:101660005445C5DB012E11D1144900205C46174AB0
:101670000B6809E093F8B26054F8201006F00306F6
:10168000314122F81010401CA842F3DBBDE8F88F6E
:1016900010B50446002003F0F4FA022003F0F1FA3A
:1016A000E00701D0FFF780FF022003F005FBBDE853
:1016B0001040002003F000BB1C031000D0021000FB
:1016C0004C021000F102100045150000823B012081
:1016D00010B51C4C40F2FF112068FFF781FE216815
:1016E000C1F8FC07FFF74CF800213F200EF1B0FADB
:1016F000FFF746F82168BDE810403F234FF4007221
:101700001148FFF782BD10B540F2FF310F48FFF7D7
:1017100067FE0E49C1F8FC0FFFF732F800213D20AB
:101720000EF196FA00213E200EF192FAFFF728F80A
:10173000BDE810403D234FF4806204490448FFF7A0
:1017400064BD0000D0021000F0EF0300480001204B
:10175000F0CF030030B41DC84F4981E81D000121BE
:1017600030BC002003F0DCB910B5002003F089FA8A
:10177000FFF7BFFB00F064F80446FFF7D0FB012C35
:1017800004D13C224549A020FFF783FC002003F050
:1017900093FA012010BD10B5FEF718FFBDE8104008
:1017A000822002F079B82DE9F047002003F069FAB1
:1017B00000253B4F4FF0360A6E1EA846E8B2FFF7F1
:1017C00072FC0020FFF749FB3C683868A042FCD05F
:1017D0003868A042FCD133496420FEF7FFFEFEF7D3
:1017E000A2FF81463868A042FCD03868A042FCD1F4
:1017F000FEF799FF0446FFF768FBFEF7E7FEA9EB4B
:10180000040080B2B0EB0A0001D4014600E041427E
:10181000B14204D2002800DA40420646A8466D1CB8
:101820006DB2202DCADB1D4908F0FF00743981F824
:10183000B000FFF738FCBDE8F047002003F03CBAE9
:10184000FEB50025684602F00FFD17480090032002
:10185000114E8DF804000446684602F009FD00228E
:1018600002AB0121104603F0ABF90121002003F087
:1018700086F9307838B1641E01F0FBFF002C05D0EA
:10188000EADC2846FEBD4FF00105FAE74FF0020002
:1018900002F0E3FCF5E7000090031000BC0001201B
:1018A000981B0022471700000517000030B41DC820
:1018B0008E4981E81D00012130BC002003F030B9C1
:1018C0002DE9F84F8A48006810F86C4F407844437F
:1018D000FEF763FF85486421103003F099FB322145
:1018E000844803F073FB3221834803F06FFB814887
:1018F00042F21071323003F069FBDFF8F8A10020EA
:10190000AAF1320A47F6FF71AAF1320BCA4304E08A
:101910002AF810102BF81020401CA042F8DB774862
:1019200002F0A2FC7549012000250871DFF8CC9176
:1019300003267349DFF8B4810027C9F80010484630
:1019400002F096FC00226B460121104603F038F9A4
:101950000121002003F013F998F80000C0B101F054
:1019600088FF761E002E16D0E9DCBFB36148D8F898
:10197000041005FB04F200F13200DFF8708100EB87
:1019800042034FF0000056465F4608F1100823E07E
:101990004FF00107E9E74FF0040002F05EFCE4E7D6
:1019A00031F8102023F8102058F8202031F910C009
:1019B000624448F8202031F9102037F910C0624500
:1019C00001DD27F8102031F9102036F910C06245EA
:1019D00001DA26F81020401CA042E1DB6D1CC82D66
:1019E000A4DBDFF808810020C821424D52465B4647
:1019F00008F110080EE033F9106032F91070F61B90
:101A0000761025F8106058F8206096FBF1F648F83B
:101A10002060401CA042EEDB364F0020364E3237AD
:101A2000894615E0002258F82030114601FB040CCD
:101A300037F91CC0BCEB030C01D5CCF1000C491CE0
:101A40006244C829F2DB92FBF9F126F81010401C21
:101A5000A042E7DB002707E036F9172035F9171019
:101A6000F8B202F01EF97F1CA742F5DBBDE8F84F83
:101A7000FEF786BE2DE9F84300248DF80040FEF7FE
:101A80008CFE002003F0FDF8194D286890F86B00DB
:101A9000FFF759FA2F680025A1464FF00108A1373A
:101AA0000024785D08FA04F68DF8009006400DD009
:101AB000224629466846FFF795FA9DF8000020283F
:101AC00004D132462946052001F0E8FF641CE4B247
:101AD000062CE6D36D1CEDB2052DE1D3002003F0FA
:101AE000EBF8FEF74DFEBDE8F8830000A003100000
:101AF000D0021000AC100120EE370120540210007B
:101B00005D18000010B504460221002003F008F81B
:101B10000F48046010BD08B50E48FEF752FE0022C3
:101B20006B460221104603F04BF80221002003F01F
:101B300026F809485522016805480A71006848716D
:101B4000020A8A71020CCA71FEF7EBFC08BD0000A4
:101B50005C021000B51A0000D402100008B5002481
:101B6000DFF85881564F4FF40049264600226B4655
:101B70004146104603F024F80098800319D5FEF77B
:101B800045FC504804680660FEF73EFCE00701D0C3
:101B9000FFF709FEA00701D5FFF7E6FD00231A466F
:101BA0000121022002F064F84FF40031002002F01D
:101BB000E6FF0098000411D500256D1CEDB2FFF77B
:101BC000D3FD01286ED0032DF7D900224946082005
:101BD00001F064FF4946002002F0D1FF00980005A3
:101BE00010D53948046806602046FFF751FD4FF4D0
:101BF0000061002002F0C3FF0023E1B21A46062074
:101C000002F036F80098C0040CD5FFF784FF0023DB
:101C100001221946022002F02BF84FF480510020D7
:101C200002F0ADFF0098800406D5FFF751FD4FF498
:101C30000051002002F0A3FF0098400406D5FFF7F2
:101C400062FD4FF48041002002F099FF00984003AC
:101C500011D5386890F8A000C0070CD0FFF70AFF34
:101C60004FF48021002002F08AFF00231A46194613
:101C70000C2001F0FDFF009800037FF577AF386876
:101C800090F8A0008007F8D5FFF71AFE4FF4002166
:101C9000002002F074FF00231A4619460E2001F0BE
:101CA000E7FF63E70120FFF7F3FCE1B20023C4F391
:101CB0000722082001F0DCFF8CE7000003F80F008A
:101CC000D0021000EC021000E802100010B58143B1
:101CD000C80711D06448016841F0010101604FF468
:101CE0000061002002F01CFF01220023BDE810402B
:101CF0001146052001F0BCBF10BDFEF7F6BC10B5C3
:101D0000FEF7F3FC0121BDE81040084602F008BFD1
:101D10005649012805D0022805D0032805D1042002
:101D200002E0022000E003200870704738B5002070
:101D300002F0A7FF4E48006810B1FFF7E9FF01E08D
:101D400000F0CCF949484B490078022813D0032809
:101D50000ED0042812D001240025FEF7DAFE00B1CF
:101D600001256946032002F01AFF009858B909E0DE
:101D70000868847AF0E70868447AEDE70868B0F804
:101D80000B40E9E715B1142C00D2142420463A493F
:101D9000FEF7B3FC0324394D00F022FA012807D1E5
:101DA000287858B1641E01F064FD002C0DD0F3DCDE
:101DB000BDE838404FF0000002F07EBF30480168B7
:101DC0003048006800F01CF9F2E7032002F045FA01
:101DD000EEE770B52C4804682C490D680C6095EA54
:101DE000040F27D0214E2DB1A4B121462846BDE8CD
:101DF00070406BE7022030701E48006800790007D1
:101E000001D40420307021462846FFF75FFFBDE86B
:101E100070408BE7FEF769FC0121084602F0AFFE37
:101E20000120307021462846FFF750FFBDE8704082
:101E300000F0F7B870BD10B5FEF757FC0121084659
:101E400002F09DFE09490420087000F0B1F8BDE8D9
:101E500010406BE710B5FEF748FC0121084602F080
:101E60008EFEBDE8104061E7E8021000700210002D
:101E7000E0021000D0021000AF1C0000140410009B
:101E80007C02100078021000D802100074021000CA
:101E90002DE9FC5F0E4600281BD05549097804291E
:101EA00017D1002A15D1DFF84C91DFF84C81534D42
:101EB000D9F800109246097A49070ED5A978491C2D
:101EC000C9B2A970032906D8018808EB460020F89A
:101ED000021CBDE8FC9F85F802A0032002F0D1FEA1
:101EE000454801906C78B5F904B02878274640B988
:101EF00041480F235A460094801D019902F0F0F8E2
:101F0000002734B93C4A5B46921D901D019902F0AE
:101F1000D8F839496F700C31B5F90420B5F906309D
:101F2000002007E031F910409C4201DD012404E06B
:101F3000401CC0B29042F5DB0024032002F0BCFE3E
:101F4000D9F8000090F8E307DA2823D1D8F8001078
:101F5000C8F81210B8F80410A8F81610D8F806102F
:101F6000C8F81810B8F80A10A8F81C10D8F80C1007
:101F7000C8F81E10B8F81010A8F822101E48C8F8AB
:101F800024A0C8F828A01230A8F82CA04682A9786E
:101F90008182C4822C70002C9BD0FFF7AEFEBDE87E
:101FA000FC5F0121084602F0BBBD14480078704771
:101FB000124A012050700F480068017A4B0790F8D0
:101FC000711002D590F86C3001E090F870305943F0
:101FD0009180B0F84A00D0800021074811709170BC
:101FE000C1600182C0F8061041817047E0E700003F
:101FF00070021000D0021000203801206002100092
:1020000070B5054630480C46224690F90D102F4811
:102010004068FFF73DFF21462846BDE8704000F0CC
:1020200014B810B5032002F02CFE4821284802F015
:10203000EFFF274901200870032002F03DFE012137
:10204000BDE81040022002F06BBD2DE9F041DFF841
:1020500084800746002698F800000D4604282CD0FE
:1020600047EA0504032002F00CFE194A174B97813A
:1020700015619868506098F8000004281FD0FF216F
:1020800011751070E0070DD01348016811F86C0F3E
:1020900049784843906042000D485968163002F074
:1020A00016FF0126032002F007FE002E09D0BDE82E
:1020B000F0410121022002F033BD0C46D2E7197B2A
:1020C000DEE7BDE8F08100005804100014041000A1
:1020D0009C04100070021000D00210002DE9F041A5
:1020E0007A4C0026DFF8E88120780227794D042811
:1020F0000ED000F0D5FB012819D07748237802686C
:102100000320022B517B10D198F8003093B113E0DB
:10211000FFF74BFF012803D098F80000012804D1F5
:102120006E49277001202E600870BDE8F08127708D
:102130002E60FAE7917B0420127AD30701D192072F
:10214000F3D52A68521C2A608A42EEDD2E60207088
:10215000EBE730B41DC8624981E81D00082130BC9E
:10216000012002F0DDBC2DE9F0415B48002400684D
:10217000C17BC90732D05B49564E27460978C9074B
:1021800027D0DFF84881012498F8001002290BD0ED
:1021900004290BD0857C00F083FB012808D052482D
:1021A000007801280BD00EE0457CF4E7C57CF2E70F
:1021B00098F80000042806D00024776006E098F81C
:1021C0000000022807D07068401C70607068A84248
:1021D00003DD776002E07760F8E700242046A4E79B
:1021E0002DE9FE4339483F4D012600783F4FDFF887
:1021F0000081032816D00428684610D0002402F07D
:1022000033F8FFF7B0FF2978C90700D0012440EA6E
:102210000401C90716D02E49097801B310E000F077
:102220002EF812E06846002402F01EF8FFF79BFF2C
:102230002978C90700D0012440EA0401C90701D068
:102240008DF804603860C8F800402A48009068465D
:1022500002F00EF8012806D00020BDE8FE8302211E
:102260008DF80410EEE702AB00220821012002F0F5
:10227000A7FC0821012002F082FC0120EDE770B5E7
:102280000446002501F0F0FFFFF76DFF1249C30778
:102290004FF0020205D00968C97B89070FD50421D8
:1022A0000BE0104B1B78DB0700D00225AB0707D5EE
:1022B0000968097A490702D50521217100E02271D8
:1022C0000A4908600A48056070BD000070021000ED
:1022D000F102100068021000D00210008402100009
:1022E0001404100074021000F00210007C021000B0
:1022F00078021000032100001C4808B500210122CB
:10230000416002708160C160491E104602F037FCD6
:10231000FFF76CFE6B4600221721012002F050FCF3
:102320000098800705D5FFF754FD0221012002F037
:1023300026FC0098C00705D00121084602F01FFCCA
:10234000FFF7F4FC0098400705D50421012002F0B6
:1023500016FCFFF770FD0098C006DBD510210120A8
:1023600002F00DFCFFF776FDD4E7000070021000CC
:102370003221504802F02ABE10B50C46C00716D0D4
:1023800000F08EFA002812D14B480068C07B80070D
:1023900003D54A480078042804D02046BDE8104000
:1023A00000F006B82046BDE8104000F035B810BD7A
:1023B0002DE9F04740494FF0010A3E4E09680A7C7A
:1023C000B1F914C0B1F916703D4902F00F04C4F11F
:1023D0001005096889460AE036F9112030F91130F4
:1023E00002EB0C08984515DBD21B9A4212DC491E01
:1023F000F2D2BAF1000F0DD0494609E036F911309A
:1024000030F91120634302FB0532121126F8112026
:10241000491EF3D2BDE8F0872DE9F04F2649294C3B
:102420004FF0010E0A68DFF88CB094F90040117C7F
:10243000B2F914A001F00F0692F86D10C6F1100861
:10244000B2F916900B4614E093FBF1F7C3EB440589
:1024500001FB1737EDB2FFB23BF9155030F9177099
:1024600005EB0A0CBC4522DBA5EB0905BD421EDCD1
:102470005B1E012BE8DABEF1000F18D0DC4614E039
:1024800092F86D50C1EB440391FBF5F705FB17156E
:10249000EDB2DBB230F915703CF91350754307FB10
:1024A00008552D112CF81350491E0129E8DABDE812
:1024B000F08F0000823B0120D00210009402100037
:1024C00098021000950210007C480021A0F801102D
:1024D00070472DE9F05F8346924689460026022028
:1024E00002F0CFFB764F754DB046386805F1010418
:1024F00090F8B010C9070FD090F86D3090F86C20AC
:102500007049584600F083F80646012801D02EB1E4
:102510002EE0102028702BE084F800803B6893F8B0
:10252000B000800724D5002248460AF0FF0193F846
:102530005F60174607E0B14205D030F911C093F84B
:10254000BC80C44502DC491EF5D237B139F916000A
:1025500093F8BD10884200DD012293F8BE10601C84
:1025600000F045F80646012804D11120287001E04A
:1025700084F80180022002F09FFB3046BDE8F09F06
:102580002DE9F0410D46074601292DD14C4C167816
:1025900000201070206890F8B100C00710D0022011
:1025A00002F06FFB4848394600684200454802F097
:1025B0008EFC464801210170022002F07DFB09E0FB
:1025C0004348016841F0010101604FF400610020BF
:1025D00002F0A6FA20683246012190F8B10000F01E
:1025E0000103052001F044FB2846BDE8F08110B549
:1025F00000231C4642B10278521CD2B202708A42B9
:1026000003D90470012300E00470184610BD2DE9C1
:10261000FF4F83B00020471E01902948FD039A46D2
:10262000006800904FF0004C2C46B0F9B3900022A7
:1026300023E0049902FB0AF001EB400E039901EB41
:10264000400B0021084610E03BF910603EF91030C5
:10265000AE42A3EB06080FFA88F8414400DD354688
:10266000A34200DD1C46401C80B25045ECD38C4593
:1026700001DA8C4657B2521C92B205988242D8D3E6
:1026800067B1012F02D0022F04D007E00098B0F903
:10269000B50002E00098B0F9B7008146CC4503DDF3
:1026A000AC4201DD012001900098019A90F8BB1026
:1026B00007B00248BDE8F04F401C98E780021000C8
:1026C000D0021000823B012098021000840210000A
:1026D000E802100010B5F94C206890F8940001074A
:1026E00015D500F0070002F048FD20680022012106
:1026F00090F8940000F00700FEF758FA20680022D6
:10270000114690F8940000F00700FEF765FA206883
:1027100090F89400010615D5C0F3021002F02DFDCB
:1027200020680022012190F89400C0F30210FEF707
:102730003DFA20680022114690F89400C0F3021080
:10274000FEF74AFA206890F89500010715D500F0C9
:10275000070002F012FD20680022012190F8950088
:1027600000F00700FEF722FA20680022114690F8D8
:10277000950000F00700FEF72FFA206890F895000A
:10278000010615D5C0F3021002F0F7FC2068002204
:10279000012190F89500C0F30210FEF707FA2068B7
:1027A0000022114690F89500C0F30210FEF714FACB
:1027B000206890F89600010717D500F0070002F096
:1027C000DCFC20680022012190F8960000F0070050
:1027D000FEF7ECF920680022114690F89600BDE85B
:1027E000104000F00700FEF7F7B910BD10B5B44C6B
:1027F000012019212070B34802F00AFCB1483221AF
:102800001A3002F0E3FBAF4832214C3002F0DEFB1D
:10281000AC490020091F0860E060A0606070BDE85E
:1028200010404FF49671A84802F0D0BBF0B5A34811
:10283000A64B02680020186058601881C3F80A008F
:10284000C3F80E0002F13E0102F14604588203F182
:102850000A060AE031F8105023F8105031F81050F1
:10286000275CED1B26F81050401C92F86C508542F6
:10287000F0DCF0BD9148006890F8801069B1490023
:1028800010F88C2F521C40784A43C2EB022100F012
:102890001F0001418A48C18070470121F0E770475D
:1028A0008748C068002800D00120704730B5012259
:1028B000874B0CE000EB420531F8124025F8024C42
:1028C00001EB420434F8024C20F81240921C1C68C0
:1028D000A242EFD330BD2DE9F04F794D4FF0010A00
:1028E0000AFA01F6AD687B4F2E407B4DDDE909B950
:1028F0004FF00008DDF82CC02D783F68444602D028
:10290000012D09D00CE0012D00D1FC8EBCF1010F8E
:1029100000D06DB96D4C09E0FC8E3F8FE41BA4B272
:10292000BCF1010F00D01DB9684C0A3434F81140D5
:102930006249096891F83A10CF0730F9121027D090
:10294000BCF1000F03D0B9F1010F06D00AE0B9F1D4
:10295000010F07D10EB9012D04D030F813500D44EA
:102960002DB204E030F913508D4200DC0D46BBF16E
:10297000010F0AD14EB1BCF1000F06D1A14204DA19
:1029800030F91300A04200DA0025A54207DC0CE074
:1029900076B1A14209DA30F91300A04205DA0AFA49
:1029A00002F00AFA03F848EA00084046BDE8F08F52
:1029B000A142F4DC30F91300A042F0DCF5E7F0B4FA
:1029C0003E4E0A4600213568146895F85F30A70727
:1029D0000AD030F9137095F860503D44002D03DDA6
:1029E00024F0030111600121146814F00C0F0BD0C6
:1029F000376830F9135097F861703D44002D03DDBE
:102A000024F00C04891C146014F0300F0BD030F942
:102A10001300336893F862301844002803DD24F073
:102A20003000091D1060306890F8E307DB2804D1FE
:102A3000F0BC0022FC2001F003B8F0BC7047F0B5F8
:102A40000125059F9D400C684FF0010214EA050620
:102A500002FA07F201D114420DD030F9177030F9A3
:102A60001300874207DD0EB1AC430C60144202D064
:102A700024EA02000860F0BD2DE9F0430E46074647
:102A800000248DB0651E04213046FEF7C3FCC0B2A1
:102A9000DFF82890012858D13421684602F0B8FAAE
:102AA00039466846FFF702FF0948A446E84607781A
:102AB0002D0D61466246604619E00000D00210000C
:102AC000840210005038012000EC01202404100082
:102AD00098021000D4021000343B012038F9103065
:102AE000634502DD03FB00111A44401CC0B2B8422A
:102AF000F4D37F1E82FB072381FB050102F0C3F99B
:102B0000002800DA0020691E884200DD084605B270
:102B10003068C10709D0D9F80010B1F84E10A942A9
:102B200003DD20F00100641C306041070DD5D9F8A9
:102B30000010B1F85620AA4203DCB1F85810A9429F
:102B400003DA20F00400241D3060D9F8000090F86A
:102B5000E307DB2807D10DB02A462146BDE8F04344
:102B6000FD2000F06DBF0DB0BDE8F08301460020F0
:102B70008A0700D0012011F00C0F01D040F00200B4
:102B800011F0300F01D040F004007047F8B5FF4C51
:102B900006460D46206890F83A00400702D53046B8
:102BA000FFF70DFF206890F83A00800717D5012045
:102BB000002300901A4629463046FFF740FF0220C6
:102BC00000900323012229463046FFF738FF0520F5
:102BD00000900423022229463046FFF730FFF8BD5B
:102BE000FEB50C4601250095CDE9015407460523A5
:102BF00004220221FFF76FFE0095CDE9015406463D
:102C00000022012311463846FFF765FE40EA06051B
:102C100000200090CDE9010403230222012138465F
:102C2000FFF759FE2843C0B2FEBD2DE9F0410C4626
:102C300001463222D64802F04AF9D5483222D54917
:102C4000323002F044F9D2483222D349643002F0E3
:102C50003EF9D149CE4832223231963002F037F96E
:102C6000CD4A0020FF231E3A4FF0010E1668CB4AD2
:102C70000746C749156814E00EFA00F2224201EB3C
:102C8000400C02D0ACF8C83001E0ACF8C870324259
:102C900001EB400202D0A2F8FA3001E0A2F8FA708B
:102CA000401CA842E8D3BDE8F0812DE9F8438146F5
:102CB000BB480027884606780770B748322196300F
:102CC00002F084F9B14DB54C286890F82A10C90774
:102CD0000AD0009690F82B00494600F00F03208898
:102CE00002B2AD4801F0FCF9022001F0CAFF2088D1
:102CF000A94900B200904346A64A01F1960001F0AE
:102D000083F9022001F0D8FFA34932229631A1F1C4
:102D1000320002F0DCF82868A24EC07B000711D513
:102D2000A148007801280DD1307858B920889A49F7
:102D300000B200909D48963102680846938E243276
:102D400001F068F82068944942009631A1F16400CE
:102D500002F0BDF8307858BB286890F82A00400788
:102D600007D58D4922786431012301F1320000F04A
:102D7000B8F9286890F82A1089070BD590F86D10DB
:102D80000091854990F86C3090F82C2096310846D7
:102D900000F054F9804932229631A1F1320002F05C
:102DA00096F87D49484664312268FFF792FB074652
:102DB0003846BDE8F8832DE9F0410025774B0646FB
:102DC0002C46681E2A46AE46DFF8D4C11F680BE0C9
:102DD00036F912308B4201DCCB4204D5012536F99D
:102DE000124050B203E0521CBA42F1D38DB19CF8AC
:102DF0000110491CC9B28CF8011032290BD9C3B299
:102E00008CF801E0E2B2C4F30721ED2000F030FFBE
:102E100001E08CF801E0284645E75C4A10B51268ED
:102E200004460020B2F81920891A0BB25B490968E0
:102E300006E034F911209A4201DCDA4200D5012083
:102E4000491EF6D210BD70B5504D024600242868C8
:102E5000C07B40071CD51046FFF7DFFF012817D1C4
:102E6000FDF7D4FA524C206840F002002060FDF7D4
:102E7000CBFA4FF40041002001F052FE286822787E
:102E80000121C07BC0F38003072000F0F1FE012484
:102E9000204670BD10B5424CA078002805D0E078DF
:102EA00020B1401EE070207910B910BD01202071C2
:102EB000394803211E38007800F00AFF0020A07076
:102EC000207110BD30B53649304B00228D681B682B
:102ED000002D14464FEAC07505D07DB185070DD58C
:102EE0008D782DB10AE04DB1850707D58C7005E0CE
:102EF00001258D700C7193F89750CD7010B18C78BE
:102F000034B901E08C700C71024693F89700C870D8
:102F1000104630BD2DE9FC4781460020009001900D
:102F2000244890F900401E4E4846B6F90610FFF7B7
:102F30008AFF01287ED0B6F906104846FFF73BFF0E
:102F4000012879D021464846FFF7AFFE0446012804
:102F500072D01148184ADFF8348064301060D8F815
:102F60000010104F154DC97B090708D50E49097887
:102F7000012904D1397811B9A0F13201116028601A
:102F800000211068FFF72CFE009019E0D00210001D
:102F900000EC0120823B01206A38012098021000D9
:102FA00084021000F0021000343B0120D402100013
:102FB000EC021000E4021000AC021000A8021000A5
:102FC00060B1387850B901212868FFF709FE0099EF
:102FD0000840009069462868FFF7D8FD0098FFF781
:102FE000C5FD0190D8F8000090F83A00000703D51D
:102FF00001A92868FFF740FD0322B168019800F09D
:10300000ACF8764D2968884207D02860C0B2FFF737
:1030100059FF0146287800F05BFEFFF73BFF704840
:103020000078042803D048460199FFF7FEFD286880
:10303000B06000E000E02046BDE8FC872DE9FF4FCE
:103040009146864600250D9F46E005FB07F0019955
:10305000012247F6FF7C01EB40066FEA0C040EEB01
:10306000400B13460021C9F1000A16E036F91100A1
:1030700048450FDA50450DDD844500DD8446844225
:1030800000DA0446002802DA4FF0000202E001DD17
:103090004FF0000301F1010189B2B942E6D352EACF
:1030A000030009D012B1012A04D004E0012B02D19F
:1030B000204601E023B1002041000BD0002107E0B1
:1030C0006046F9E736F81120121A2BF81120491C36
:1030D000B942F7DB6D1CADB203988542B5D3BDE8AC
:1030E000FF8F2DE9F04F00259B469AB0531E03F049
:1030F000FF0C2C462B460DF1340AE94612E031F95B
:10310000136035445E1C374695FBF6F629F81360CC
:10311000ACEB03065B1C31F91680444494FBF7F7D3
:103120002AF816709342EADBBBF1010F01D1921E1F
:10313000D2B24C4655460CE034F9123035F91260E3
:10314000334431F8126003EBD373A6EB630320F82A
:103150001230521EF0D21AB028E42DE9F047DFF801
:10316000849005461D48D9F80C301F4C85EA0308A9
:103170001A4F002300684FF0010A3F1D266820E027
:103180000AFA03F414EA080F10D02C420AD001EA1C
:10319000050C5FEACC7C02D096F83CC004E096F8BF
:1031A0003BC001E096F83DC007F803C017F903C023
:1031B000BCF1000F0BD0ACF1010C07F803C05B1C95
:1031C0001BB29342DCDBC9F80C50BDE8F0872C42FF
:1031D00001D02043F3E7A043F1E700004C38012081
:1031E0007002100084021000D0021000354808B5AB
:1031F0000021C160816041600121017032491420C9
:103200000870FFF7F3FAFFF7B3F8FFF75DF9FFF780
:1032100031FB6B4600220121022001F0D1FC009815
:10322000C007F6D00121022001F0A9FC00F001F84E
:10323000EFE770B50025032001F023FD00F01EF834
:10324000204C207BC00703D02069FFF763FE0546B2
:10325000A06848B1022001F014FD2169A068FFF7C1
:103260008BF8022001F028FD184A29462069FFF753
:1032700087F9BDE87040032001F01EBD70B5114C08
:10328000134DE068B5F90C1080EA0102D20708D0AE
:10329000C90702D0FFF7AAFA03E0C00701D0FFF781
:1032A000FEFAB5F90C00E0602869A060A8686060CB
:1032B00007481630206128782070287D6070054806
:1032C000606170BD94021000E402100080021000E2
:1032D0009C0410009C380120094C00202060401CF8
:1032E0002060FDF75AFA00F019FEFDF729F908B938
:1032F000FEF70FF9FCF76EFF01F0FCF92068EEE72E
:10330000B0021000C44900200860C4490860C449E4
:1033100008607047D0214DF6C062BA2000F0BEBBF5
:1033200070B54FF40063984202D2BE4C246807E0A7
:10333000A0F5805080B24FF4805398420CD2BA4C22
:1033400085189D4200DD1A1A002303E0CD5C1E188B
:103350005B1CA5559342F9DB70BDB0F5805F04D2CC
:103360000A460146AF48006808E0B0F5FE5F07D3A3
:10337000A0F5FE5080B20A460146AB4800F0ABBB58
:10338000704700F000BF10B54FF40051002000F06E
:1033900035F90023BDE810401A461946032000F015
:1033A00067BC10B54FF48041002000F027F90023DE
:1033B000BDE810401A461946042000F059BC964951
:1033C0000A6882430A600221012000F017B992497D
:1033D0000A6802430A600221012000F00FB9FDF7DC
:1033E00078BBFDF751BB10B5C00711D08F48002343
:1033F0000222016841F0010101600121052000F075
:1034000037FCBDE810404FF40061002000F0F6B832
:1034100010BD10B50324FCF7F9FF85480460FCF7E4
:10342000F3FF002301211A46084600F021FCBDE805
:1034300010404FF40031002000F0E0B810B5002338
:1034400001221946104600F013FCBDE810404FF46D
:103450008051002000F0D2B80421012000F0CEB845
:10346000012802D108787349087070476C4A00231C
:103470000128136005D1087810211060012000F0A8
:10348000BDB870474FF48021002000F0B7B84FF46A
:103490000021002000F0B2B862480021006890F8D6
:1034A0006800C00711D064480068827A12B1FF2A10
:1034B00003D00AE0C27A1AB107E0C27AFF2A04D127
:1034C00096218172A521C172012100231A46102084
:1034D00000F0CEBB584800210B4600680A468172B6
:1034E000C172202000F0C4BB10B50978534C0020F5
:1034F00021B1012121705249087000E020700120A3
:10350000FFF771FF00232178BDE810401A469A208A
:1035100000F0AEBB10B5494C2278002A11D0464AC3
:1035200000EBD070136820F0010203F1340001F0C9
:10353000CEFC00232178BDE810401A469C2000F004
:1035400097BB10BD3D4A1278002A0BD0012809DC38
:1035500039480978002300681A4680F83A109D20FF
:1035600000F086BB704770B5344C2278A2B1324D62
:1035700000EBD07626F001022B6803F1240001F065
:10358000A6FC29687008002348842178BDE87040B3
:103590001A469B2000F06CBB29480078002811D106
:1035A000204B284A284C1B6808E031F8105022F8BC
:1035B000105031F8105024F81050401C93F86C5003
:1035C0008542F2DC70BD70B51B4A4D78431E14680D
:1035D0000A781D445434202D02DBDBB2FF2108E0C1
:1035E000A318421E1846491C01F071FC00231A461C
:1035F0000121BDE87040992000F03ABB38B50C4677
:10360000054601F08DFA6946284601F0C8FA009A8D
:103610002242F8D138BD0000D8021000DC021000B0
:10362000E0021000D002100048000120E802100063
:10363000EC021000E4021000D4021000F0021000AE
:10364000343B0120240410002E04100010B520216A
:10365000494801F0BBFC4848FDF742FA4649401E84
:1036600011F8012BA2F190031F2B05D8434A52F801
:103670002320BDE810401047B82A21D00DDCB02A25
:1036800013D0B22A27D1032825D108888A78BDE82B
:10369000104040BA1146FFF760BEFB2A17D0FC2A43
:1036A00019D1BDE81040FFF77CBE022813DD31F8C8
:1036B000022BBDE8104053BA821E1846FFF730BEF9
:1036C000022808D10888BDE81040FFF75ABEBDE8BF
:1036D0001040FFF758BE10BD0120FFF778BE012053
:1036E000FFF76DBE0120FFF77EBE00F03CBA244913
:1036F000022008700120FFF776BE214903200870E0
:10370000FFF794B810B51E491E4C012008702068C0
:103710000078A52802D0012000F0B0F840F2FF1197
:103720002068FDF75DFE2168D1F8FC17814202D0C8
:10373000022000F0A3F840F2FF311348FDF750FEDD
:103740001149D1F8FC1F814206D02068007980071A
:1037500002D4032000F092F8BDE810400120FFF7EA
:1037600042BE07490020087006480068007A8007BA
:1037700001D5FFF771BE704738041000AC5500004A
:10378000F1021000D00210004800012008B5FFF738
:10379000B9FD00F0CBF91B4C20680079800701D5FA
:1037A000FFF737FE20680079C00701D0FFF794FFCC
:1037B0002168C87B00070DD511F86C0F4978484384
:1037C00000F0FEFA104900231A4608700146C02096
:1037D00000F04EFAFFF72AF801216B460022032081
:1037E00001F0EEF90098C007F6D0FFF72FFF012196
:1037F000032001F0C4F9FDF787F9EDE7012103206B
:1038000001F08EB9D0021000343B0120304C2F4A19
:10381000C4E900210168A1604168E160816821611B
:10382000C16861610169A1614169E16181692162E8
:10383000C069606204F12800FDF77BFE01F0D9FA4F
:10384000606400F035F82249224AC1E9002070473F
:1038500010B501284FF0000205D00146BDE8104028
:10386000022000F01BB90121022000F017F900F03E
:103870001FF8012801D10220EAE7704710B504467D
:1038800001460022032000F009F9012C01D0042C8C
:1038900001D100F00DF810BD00220146062000F015
:1038A000FDB801460022072000F0F8F800F000F80B
:1038B000FCF773FF0848006890F89400010603D5F0
:1038C000C0F3021001F050FCFEE70000AF0550FA13
:1038D00000EE0120BA0110ABD002100077B585B020
:1038E0000E46BDF814401546200A40EA0420ADF803
:1038F00014004F48BDF8141000240180A0F580701A
:10390000CDE900044B480294039400681346484AEA
:10391000C0790221FDF765F808B02A463046BDE8B7
:103920007040454901F0D3BA17B581B00B46BDF8D8
:1039300004001446010A41EA0020ADF804003C48A6
:10394000BDF8041020F8021B194601F0C0FA00204F
:10395000009038480023364A0068A11CC079FDF762
:103960000FF81FBD77B585B00E46BDF8144015465B
:10397000200A40EA0420ADF814002D48BDF81410C8
:10398000002401802C48CDE900042A4802940394C5
:1039900000681346264AC0790221FDF722F808B0D4
:1039A0002A463046BDE87040234901F090BAFCF742
:1039B000D7BD08B50020ADF8000002226946FFF728
:1039C0008DFFBDF8000008BD00B587B000220121C1
:1039D0000720FDF7EBF8072001F0C6FB00204FF4AD
:1039E000FA7100BF401C8842FBDB072001F0C5FBD9
:1039F000FFF7DFFFA0F584410E3902D00120FFF769
:103A000027FFAFF2DB000190AFF22F100090AFF272
:103A1000AB000290AFF2690003900848049040F2B6
:103A20008F20ADF814006846FDF760F907B000BDBF
:103A3000343A0120D002100034390120030500007F
:103A40001CB5DB238DF800308DF801008DF80210D5
:103A5000100E8DF80300100C8DF80400100A8DF87C
:103A600005008DF80620684600F094F91CBD1CB5D1
:103A7000DB238DF800308DF801008DF80210100E58
:103A80008DF80300100C8DF80400100A8DF8050065
:103A90008DF806206846FDF746F81CBD1CB50F23BF
:103AA0008DF800308DF801008DF80210080A8DF8AD
:103AB00003008DF80420100A8DF80500100C8DF815
:103AC0000600100EBA498DF80700012008706846FC
:103AD000FDF729F81CBD2DE9FC410027064600979B
:103AE000122015460C4601978DF800001AE0200AB6
:103AF0008DF80100C4F30B008DF80240315C3044B6
:103B00008DF8031041788DF8041081788DF8051038
:103B1000C0788DF806008DF80770684600F03AF915
:103B2000241D2D1F002DE2DCBDE8FC811CB500200A
:103B3000A04900900190096810234A7889788DF88F
:103B400000308DF804008DF801008DF805208DF807
:103B500002008DF806108DF803008DF80700684606
:103B600000F018F91CBD70B588B000240094142032
:103B700001948DF80000FDF7FDFC8DF80100F220A6
:103B80008DF803008B4E28208DF804003068884D96
:103B900041788DF8051080788DF80600287880012E
:103BA0008DF80700684600F0F5F8009415200194A0
:103BB0008DF80000306890F8EC178DF8011090F83F
:103BC000ED178DF8021090F8EE178DF8031090F8AD
:103BD000EF078DF80400287880018DF8070068460B
:103BE00000F0D8F8009402A80194FDF7D4FB1B2044
:103BF0008DF800000298000E8DF801000298000C6C
:103C00008DF802000298000A8DF8030002988DF8E2
:103C100004008DF8054004988DF80600287880018E
:103C20008DF80700684600F0B5F800941C208DF868
:103C3000000003980194000E8DF801000398000C19
:103C40008DF802000398000A8DF8030003988DF8A0
:103C5000040005988DF8050006988DF80600287870
:103C600080018DF80700684600F094F808B070BD38
:103C70001CB5504C246894F8E247A40710D50024E2
:103C80000194009416248DF800408DF801008DF801
:103C900002108DF803208DF80430684600F07AF8A1
:103CA0001CBD1CB5002300930193E1238DF8003067
:103CB0008DF80100080A8DF80200100A8DF8040042
:103CC0008DF803108DF80520684600F063F81CBDE0
:103CD0007CB5384E05460C46306890F89300C00716
:103CE0000CD0002000900E2101908DF800108DF86E
:103CF00007008DF80150684600F04CF8306890F8E5
:103D00009400010708D5E10700F0070002D001F098
:103D10002BFA01E001F031FA306890F894000106C6
:103D200008D5A107C0F3021002D501F01DFA01E089
:103D300001F023FA306890F89500010708D569076B
:103D400000F0070002D501F00FFA01E001F015FACA
:103D5000306890F8960001071BD5174909780029AB
:103D600017D01649097800294FEA847109D0002933
:103D70000FD1A9070DD1BDE87C4000F0070001F08C
:103D8000FCB90029F5D0BDE87C4000F0070001F047
:103D9000EBB97CBD10B50446012000F072FF20464F
:103DA000FCF7C1FEBDE81040012000F085BF000017
:103DB000B4021000D0021000F102100088021000BE
:103DC000F0B51D49074601200B68598C01B303F17A
:103DD000340603F12404B51C00214FF6FF7C383370
:103DE00008E034F811200AB1624501D1002003E057
:103DF000491C89B2B942F4D3318809B1FF2900D1F5
:103E00000020298821B1FF2902D01A88914200D2CE
:103E10000020F0BDF0B50024059E0AE031F91450F1
:103E200032F814705D4395FBF7F520F81450641CCC
:103E3000A4B2B442F2DBF0BDD402100070B546214A
:103E40002C4801F0C3F82B4CA6202B4D20804FF2BC
:103E50002820608028684178217180786071FDF7A2
:103E600085FBE080FFF7A5FD2081286890F86C10A5
:103E7000217790F86D1061772049E18320492184F2
:103E8000204961842049A1872049A1842049E184F7
:103E900020492185D0F8FC170A0C6285A185C18FC5
:103EA000E185B0F840102186B0F842106186B0F884
:103EB0004410A18690F8741001F0030284F83620B3
:103EC000C1F3011184F8371090F8681001F0010176
:103ED0002187114909684A8952BA628701F1220291
:103EE000E2875431A4F8421090F8690084F8440045
:103EF00070BD000000000120D0021000363B012000
:103F00006A3801209C380120CE380120823B0120F4
:103F1000BC0001204C380120D402100010B5FCF781
:103F200075FAFDF7E4FA08B1FDF7DBFABDE81040D9
:103F3000FCF76ABA10B5FCF769FAFDF7D8FA08B9C8
:103F4000FDF7C9FABDE81040FCF75EBAF0B5851A76
:103F5000DDE905471E1B75438E1A012F02D09042E2
:103F600006DD0BE0904201DC1846F0BD884201DB23
:103F70002046F0BD95FBF6F0181A04E08842F3DA0B
:103F800095FBF6F0204440B2F0BD2DE9FC4F04460D
:103F900063480B4600260768354607F58A7207F521
:103FA0008E7C125707F5927807F5967107F59A7986
:103FB00007F59E7A07F5A27B184607F5A6779A4281
:103FC00000DD10460957994200DA084682420ADCB1
:103FD0001CF90430834206DB194619F90430012527
:103FE0001AF9044008E018F90420824209DC8142F1
:103FF00007DB3B571BF90440CDE90045FFF7A6FF5F
:1040000006463046BDE8FC8F2DE9F04F98469146B4
:104010008A4605460024424E424FDDF824B027E090
:104020003AF8141039F81400081A25F8140030680A
:10403000C07BC0061AD53C480078B8B9A0B241464A
:10404000FFF7A3FF316891F8E317882904D13919E4
:1040500087F8308281F8310240B135F914104843B5
:10406000642290FBF2F0084425F81400641C24B28A
:104070005C45D5DB306890F8E30788281FD12B4ECC
:104080006FF0130530883D54401C30800024A0B2EE
:104090002946FFF77AFF3188641C24B27854491C02
:1040A0003180062CF3DB6D1C6DB23C2DEADB3088D1
:1040B000B0F50C7F07F8008001D300203080BDE808
:1040C000F08F70B5002408E031F8145032F8146015
:1040D000AD1B20F81450641C24B29C42F4DB70BD6C
:1040E000F0B4049C012C04D01BB1C3F110060024D1
:1040F00012E0F0BC520000F0EABE30F9145031F981
:1041000014705D4307FB0655EF1705EB17752D116E
:1041100020F81450641C24B29442EEDBF0BC7047CB
:10412000D0021000B43B0120F0021000B6021000D3
:104130000FB42DE9F05F0025DDF874A08B468146B1
:104140002E464FF0010808FA06F7002407EA0B078D
:104150006FB108FA04F010EA090F08D03246214680
:104160000C9800F0B9F90AF805006D1CEDB2641C5A
:10417000E4B2052CECD3761CF6B2052EE3D3BDE8F1
:10418000F01F5DF814FB10B5044650212B4800F0D9
:104190001DFF2B4A1178491C1170A00504D5BDE8FC
:1041A0001040264800F001B810BD2DE9F04104464A
:1041B00090B0A52020704FF40070A4F8010000F02A
:1041C00092F8207100F08AF8607100F082F8804661
:1041D00000F07AF805461B4800680179552904D19A
:1041E000D0F8050020F07F40A060174E392206F17C
:1041F000740796F8B000207304F130000F90391D59
:10420000684600F0A9FE002229464046736FFFF77A
:104210008FFF04F110000F903922391D684600F01D
:104220009BFE012229464046736FFFF781FF044839
:104230000078E07010B0BDE8F0810000008001203F
:10424000B8021000D40210004800012010B500F0A0
:1042500001F91B490020086010BD10B5FFF7F3FA03
:10426000BDE81040FCF735BC00210160416070479B
:1042700010B5017999B1134900220A604A608A6039
:10428000CA600F49D0E90020C1E90120081D00F0F3
:104290001FF90B48001D00F0B3F9012010BD0020EC
:1042A00010BD10B50749064C087020688860201DB5
:1042B0000168044888472068401C206010BD000049
:1042C000BC02100058041000FD48006890F86A0015
:1042D0007047FB48006890F86B007047F84800682A
:1042E00090F86C007047F648006890F86D007047D1
:1042F00070B5040004D1FCF7ECFCF349F1484860C8
:10430000F248F34A002101701160F2480123036072
:10431000450685F8EE10F04EA0253560016013606B
:104320002046BDE87040FFF7BCBF10B5044614211D
:1043300000F06EFE0020207080206070A020A07031
:10434000FFF7C7FFE070FFF7BFFF2071FFF7C6FF61
:104350006071FFF7C8FFA071D948E279006810F8D2
:10436000771F61F38612E27110F80519490861F3AD
:10437000C712E271C18821818168E1600378217CE4
:1043800063F30001217403785B0863F34101217436
:1043900003789B0863F3820121740378DB0863F3DD
:1043A000C301217403781B0963F30411217403789A
:1043B0005B0963F34511217403789B0963F387114B
:1043C00021744378617C63F30001617443785B0876
:1043D00063F34101617443789B0863F38201617464
:1043E0004378DB0863F3C301617443781B0963F30B
:1043F0000411617443785B0963F345116174437878
:104400009B0963F386116174837863F30102E2719F
:1044100083789B0863F38202E27183781B0963F35C
:10442000C402E27183789B0963F34512E271C2789A
:1044300062F3C7116174C1780A09A17C62F30101BA
:10444000A174007960F38201A1742046BDE8104098
:10445000FCF7E1BC2DE9F0419C4800244FF0E02737
:10446000047044708470C47004714FF080764FF013
:104470000108C7F880619948A02580F800542022DF
:1044800097499848843700F067FD934808380560DD
:10449000954804608F49091DC1F80080710181F8B9
:1044A000DE80C7F8FC61FE673D229049A020FCF742
:1044B000F5FD8E48743890F8B000FCF7F4FD8C4898
:1044C000FFF733FFBDE8F0418948143000F0D4B85D
:1044D0007E49002008707047844B02EB4202743B17
:1044E00003EB820202EB410110B191F875007047B5
:1044F00091F8740070472DE9F041DFF8C4C102461D
:104500000024714D0127714BDCF80000052912D001
:10451000042949D0FFF7DDFED070FFF7D5FE1071FA
:10452000FFF7DCFE5071FFF7DEFE9071BDE8F04151
:104530001046FCF7E0BB017A490726D593F9031032
:104540000CE090F86E6007FA01FE16EA0E0F04D038
:10455000D9701979491C197102E0491C0529F0DB51
:10456000D97890F86A6007FA01FE06EA0E0616711D
:10457000577193F904606E73491CD97090F86C10F0
:10458000B14209DCDC701C7106E06C7390F86E10AF
:10459000117190F87010517190F86F00D070DCF8C4
:1045A000000090F87100C0E793F901100CE090F85A
:1045B0006A6007FA01FE16EA0E0F04D05970997866
:1045C000491C997002E0491C0529F0DB57715978A4
:1045D00010F86A6F8F403E4016714078D070DCF85A
:1045E0000000491C90F86D60967193F902602E737B
:1045F000597090F86C00B04298DC5C709C7095E744
:1046000030B5047989B0B4B12021684600F000FDCE
:104610006D4621463648FFF76EFF3549202214319A
:10462000284600F099FC0025062C10D2DFE804F0A3
:104630000F0F060D060609B0012030BD20480068A6
:1046400090F890008DF8110001E08DF81F50684639
:10465000FCF7FBFB1D49012008701F480C38056062
:104660001120410781F8EE00E5E71848007801289D
:1046700001D1FCF71EBB7047AFF28B3101601149CD
:1046800081603231C160002101740D49096811F85F
:10469000802F42744A7882744A8882828A88C282D1
:1046A000CA8802830A8942834A8982830A7B827785
:1046B000497B01F01F01C17741F288318180704749
:1046C000D0021000363B012058041000C802100030
:1046D00010050022901B0022100C022018E000E0C0
:1046E0002C56000000000220E01E0022BC00012029
:1046F0006804100010B5FCF712FFFCF741F8BDE8A4
:104700001040FFF717BC0BF1C5BA10B5FFF7F2FF69
:1047100010BD10B5FFF7EEFF10BD10B5FFF7EAFFB3
:1047200010BD10B5FFF7E6FFBDE81040FFF766B813
:1047300010B5FFF7DFFF10BD10B5FFF7DBFFBDE8D9
:104740001040FBF723BF10B5FFF7D4FFBDE81040C2
:10475000FBF75ABF10B5FFF7CDFFBDE81040FBF7E0
:104760007CBF10B5FFF7C6FF10BD10B5FFF7C2FF45
:10477000BDE81040FBF799BF10B5FFF7BBFFBDE8E0
:104780001040FBF7D8BF10B5FFF7B4FF10BD10B550
:10479000FFF7B0FF10BD10B5FFF7ACFF10BD10B5AF
:1047A000FFF7A8FF10BD10B5FFF7A4FF10BD10B5AF
:1047B000FFF7A0FF10BD10B5FFF79CFF10BD10B5AF
:1047C000FFF798FF10BD7047704710B5FFF792FFD5
:1047D000BDE81040FCF711B870477047704770474C
:1047E00010B5FFF787FFBDE81040FFF73EBF7047E9
:1047F00030B58DB04FF22820FCF797FEFCF753FE42
:104800004FF400624B494C4800F0A6FB4FF4805235
:104810004A494B4800F0A0FBFCF73CF90120FCF7AB
:1048200050F9FCF7E5FC0E246846FCF703FD0698FA
:10483000C01C65D00698401C64D00698801C61D0CE
:104840000698C4B22046FCF75DFEFCF744FEFCF778
:1048500095FE3C4C20680078A52802D00120FFF787
:104860000DF840F2FF112068FCF7BAFD2168D1F87D
:10487000FC17814202D00220FFF700F840F2FF311E
:104880002F48FCF7ADFD2E49D1F8FC1F814206D020
:1048900020680079800702D40320FEF7EFFFFCF7C1
:1048A00063F9FBF7B5FD2948274D016808795528BC
:1048B0002CD07020FEF7F0FF2846FBF732FEFCF705
:1048C00025F820680079400704D4214900200860B9
:1048D000091F0860FFF778F8FFF7B8FCFBF762FFE5
:1048E00038B1002211460120FFF7D8F80120FEF769
:1048F000AAFFFBF740FF0DB0BDE83040FDF7EABE70
:10490000312000E03020FEF7C7FF9BE7D1F805001B
:1049100020F07F45D0E710B5FBF778FDFFF768FF83
:10492000FFF78CFA00F016F8FBF76EFD00F07EF84A
:10493000012010BDF0EF030000F00120F0CF0300D4
:1049400048000120D002100000770100D4021000BE
:10495000841400227FB500F041F81F4D002405EBC0
:10496000441000F11002017F4CCACDE90261CDE98B
:1049700000230FC800F0DAF910B10220FEF791FF12
:10498000641C052CEBDB144D0024A03504EB440023
:1049900005EB800155F820008A68496800F046F967
:1049A00010B10220FEF77DFF641C042CEEDB0A4DE3
:1049B0000024D03505EBC400416855F8340000F000
:1049C0008FF810B10220FEF76CFF641C042CF1DBA1
:1049D0007FBD0320FEF765BF4C5600001A4910B595
:1049E0000120087019490020086019490860194918
:1049F00008601949086000F07DF900F00FF900F037
:104A000067F8002010BD10B5124800F024FA1049D4
:104A100008600E490968884207D00B4800780228D0
:104A200003D1BDE81040FBF7A9BC10BD10B5FFF7DE
:104A3000EAFF054902200870FBF784FC4FF0FF30C5
:104A400010BD052070470000F2021000F4021000B3
:104A5000F8021000FC0210000003100070B50D46B3
:104A60000446C1698068CC2200F0A8FAE169A06818
:104A7000084440384FF08071C163216A816300218E
:104A800041630163C1628162C0E908514FF00B319B
:104A9000C1614FF00A3181614FF0093141614FF03E
:104AA000083101614FF00731C1604FF0063181607C
:104AB0004FF0053141604FF00431016070BD8269F3
:104AC0008168914202D84068FFF783BF70470000B9
:104AD00010B54FF4B4714F4800F09AFA002010BDA1
:104AE00070B5054600EBC5014A4800EB8104FBF7B1
:104AF0007DFC0646207828B13046FBF77FFC6FF03E
:104B0000010070BD0320207000206560206204F168
:104B10001C0000F079F93046FBF770FC002070BDF6
:104B20002DE9F0410F463B49002500EBC00001EBA9
:104B300080042E46FBF75AFC8046206A38432062E8
:104B400004F11C00074600F086F90CE0216A026CB3
:104B5000114203D000F026F9012600E06D1C294621
:104B6000384600F06EF90028F0D1012E01D1FFF790
:104B70004AFF4046FBF742FC0020BDE8F08170B5DB
:104B80000D46244900EBC00001EB8004FBF72EFC2E
:104B9000216AA9432162FBF731FC002070BD70B58A
:104BA0000C461C4900EBC00001EB80050020206092
:104BB000FBF71CFC296A2160FBF720FC002070BD7C
:104BC0002DE9F0410D46134900EBC0001E4690460A
:104BD00001EB8004FBF70AFC07460F4800680564F8
:104BE000216A294203D104F11C0100F0EDF8384696
:104BF000FBF704FCFBF7FAFB216A29403160B8F1AE
:104C0000010F02D1216AA9432162FBF7F7FB0020C3
:104C1000B3E70000A4181000F402100010B54FF420
:104C2000C871324800F0F4F9002010BD2DE9F041C0
:104C3000884605462D4900EB8500174601EBC00468
:104C4000FBF7D4FB0646207830B13046FBF7D6FBA5
:104C50006FF00100BDE8F08102202070E7611422AE
:104C6000414604F10800656000F031F9002020623F
:104C700004F1240000F0C8F83046FBF7BFFB002029
:104C8000E8E770B5194900EB800001EBC004FBF7C1
:104C9000ADFB0546D4E90701814205DB144804F168
:104CA0002401006800F090F8206A401C2062284629
:104CB000FBF7A4FB002070BD70B50C4900EB800031
:104CC00001EBC004FBF792FB0546206A08B1401EC9
:104CD000206204F1240000F0BEF810B1606A00F018
:104CE00011F82846FBF78AFB002070BD0C1A100053
:104CF000F402100010B54FF42A71404800F088F912
:104D0000002010BD10B5044690F8380002280BD0E2
:104D1000204600F0A2F8022084F8380038492046E6
:104D200000F076F8FFF76FFE002010BD2DE9F05F70
:104D30008B460646314900EB06109046DDE90AA98C
:104D400011F820201D461AB16FF00100BDE8F09F58
:104D500001EB8004FBF74AFB074601202070C4E901
:104D60000165C4E90585C4E907A91422594604F17F
:104D7000240000F0ACF8002084F8370084F83800F4
:104D80006169E0602061C4E90F1020460C99FFF7CB
:104D900065FEA0602046FFF7B5FF3846FBF72EFB07
:104DA0000020D3E710B5044690F83800022809D057
:104DB000204600F052F8022084F8380010492046BE
:104DC00000F026F8002010BD70B5044690F83800B9
:104DD0000D4602280BD1204600F03FF8032084F84E
:104DE00038002946204600F013F8FFF70CFE00209B
:104DF00070BD044800684068704700009C1B1000AC
:104E0000FC021000F4021000002101600846704707
:104E100030B50A6812B10B46C46B09E00022086085
:104E2000C0E903210BE000BF02F10C03D26812B10C
:104E3000D56BA542F8DC1A68C0E903211860002090
:104E400030BD0068002201E0C068521C8A4201D0D7
:104E50000028F9D170470068704702690AB11168EB
:104E600031B96FF00400704701F10C02C96839B123
:104E70008142F9D1C968116000210161084670477B
:104E80006FF00300704710B54C1084EA530404D54A
:104E90004042C1F1000138BF491E1B4204D55242B5
:104EA000C3F1000338BF5B1E00F0D9F814F0804F47
:104EB00004D04042C1F1000138BF491E14F0004F38
:104EC00004D05242C3F1000338BF5B1E10BD032A59
:104ED00040F2308010F0030C00F0158011F8013B17
:104EE000BCF1020F624498BF11F801CB00F8013BFE
:104EF00038BF11F8013BA2F1040298BF00F801CBC2
:104F000038BF00F8013B11F0030300F02580083A98
:104F1000C0F0088051F8043B083A51F804CBA0E8EF
:104F20000810F5E7121D5CBF51F8043B40F8043B44
:104F3000AFF30080D20724BF11F8013B11F801CB79
:104F400048BF11F8012B24BF00F8013B00F801CB4A
:104F500048BF00F8012B704710B5203AC0F00B8015
:104F6000B1E81850203AA0E81850B1E81850A0E86D
:104F70001850BFF4F5AF5FEA027C24BFB1E81850C7
:104F8000A0E8185044BF18C918C0BDE810405FEA37
:104F9000827C24BF51F8043B40F8043B08BF7047B3
:104FA000D20728BF31F8023B48BF11F8012B28BFB8
:104FB00020F8023B48BF00F8012B704702F0FF03C6
:104FC00043EA032242EA024200F002B84FF0000234
:104FD0000429C0F0128010F0030C00F01B80CCF10B
:104FE000040CBCF1020F18BF00F8012BA8BF20F879
:104FF000022BA1EB0C0100F00DB85FEAC17C24BFCD
:1050000000F8012B00F8012B48BF00F8012B704776
:105010004FF0000200B5134694469646203922BF51
:10502000A0E80C50A0E80C50B1F12001BFF4F7AF9C
:10503000090728BFA0E80C5048BF0CC05DF804EB7E
:10504000890028BF40F8042B08BF704748BF20F8EC
:10505000022B11F0804F18BF00F8012B704753EA64
:10506000020C00F069802DE9F04B4FF00006002B98
:105070001FBFB3FA83F503FA05F424FA05F65E4080
:1050800012BF1643B2FA82F502FA05F4C5F1200503
:105090001EBF22FA05FC44EA0C04203556EA044CF3
:1050A0004FEA144418BF641C4FF000084FF0000989
:1050B000904271EB030C39D3002919BFB1FA81F783
:1050C00001FA07F6B0FA80F700FA07F6C7F12007F1
:1050D0001EBF20FA07FC46EA0C062037B6FBF4FC9C
:1050E000A7EB0507103F07F01F0BCBF120060CFACA
:1050F0000BFB2CFA06F644BFB3460026202FA4BFB4
:105100005E464FF0000B5BEA060C08BF4FF0010B48
:1051100019EB0B09ABFB027C48EB0608C01B06FB36
:1051200002CC0BFB03CC71EB0C01C1E70B46024632
:1051300041464846BDE8F08B13B54FF000004FF0F4
:105140000001AFF30080BDE81C4070470446AFF398
:1051500000802046FBF734F8704700000149182012
:10516000ABBEFEE726000200012181404FF0005057
:1051700010F8352F8A4302707047012181404FF0AB
:10518000005010F8352F0A4302707047441D0A5D25
:105190003F1E1D1D06080708220F052F200F0F0FA9
:1051A000020404041108031810080808000202028F
:1051B0000904020C08040404000101015A280D7BB3
:1051C00054282828090B090B2D14073E2A141414FF
:1051D00004060506170A041F150A0A0A0103030339
:1051E0000C0502100B050505000202020001010278
:1051F0000102020301020203020303040000000093
:105200001B0000802D00008036000000410000805F
:105210005A0000006C0000007700008099000080B8
:1052200082000000B4000000AF000080D800000041
:10523000C3000080F5000080EE000000290100801E
:1052400032010000040100001F010080680100001D
:1052500073010080450100805E010000B001000084
:10526000AB0100809D01008086010000F1010080FB
:10527000EA010000DC010000C70100804902008053
:1052800052020000640200007F0200800802000059
:1052900013020080250200803E020000D0020000C0
:1052A000CB020080FD020080E60200009102008037
:1052B0008A020000BC020000A70200806003000018
:1052C0007B0300804D030080560300002103008013
:1052D0003A0300000C03000017030080F90300806C
:1052E000E2030000D4030000CF030080B8030000F5
:1052F000A3030080950300808E03000089040080D2
:1053000092040000A4040000BF040080C804000050
:10531000D3040080E5040080FE04000010040000B7
:105320000B0400803D04008026040000510400802E
:105330004A0400007C04000067040080A00500000F
:10534000BB0500808D05008096050000E10500800A
:10535000FA050000CC050000D70500803905008063
:1053600022050000140500000F05008078050000EC
:1053700063050080550500804E050000C006000052
:10538000DB060080ED060080F60600008106008046
:105390009A060000AC060000B7060080590600809F
:1053A00042060000740600006F0600801806000028
:1053B00003060080350600802E060000E907008005
:1053C000F2070000C4070000DF070080A807000004
:1053D000B3070080850700809E070000700700006B
:1053E0006B0700805D0700804607000031070080E2
:1053F0002A0700001C070000070700800909008039
:1054000012090000240900003F090080480900003B
:1054100053090080650900807E09000090090000A2
:105420008B090080BD090080A6090000D109008019
:10543000CA090000FC090000E709008020080000FC
:105440003B0800800D0800801608000061080080FD
:105450007A0800004C08000057080080B908008056
:10546000A2080000940800008F080080F8080000DF
:10547000E3080080D5080080CE080000400B000043
:105480005B0B00806D0B0080760B0000010B008031
:105490001A0B00002C0B0000370B0080D90B00808A
:1054A000C20B0000F40B0000EF0B0080980B000013
:1054B000830B0080B50B0080AE0B0000690A0080F2
:1054C000720A0000440A00005F0A0080280A0000F7
:1054D000330A0080050A00801E0A0000F00A00005E
:1054E000EB0A0080DD0A0080C60A0000B10A0080D5
:1054F000AA0A00009C0A0000870A0080800D0000B4
:105500009B0D0080AD0D0080B60D0000C10D008028
:10551000DA0D0000EC0D0000F70D0080190D008081
:10552000020D0000340D00002F0D0080580D00000A
:10553000430D0080750D00806E0D0000A90C0080E9
:10554000B20C0000840C00009F0C0080E80C0000EE
:10555000F30C0080C50C0080DE0C0000300C000055
:105560002B0C00801D0C0080060C0000710C0080CC
:105570006A0C00005C0C0000470C0080C90F008022
:10558000D20F0000E40F0000FF0F0080880F000022
:10559000930F0080A50F0080BE0F0000500F000089
:1055A0004B0F00807D0F0080660F0000110F008000
:1055B0000A0F00003C0F0000270F0080E00E0000E3
:1055C000FB0E0080CD0E0080D60E0000A10E0080E4
:1055D000BA0E00008C0E0000970E0080790E00803D
:1055E000620E0000540E00004F0E0080380E0000C6
:1055F000230E0080150E00800E0E000049340000BE
:10560000853400008F36000089360000C532000066
:10561000C5320000C5320000ED330000C532000085
:10562000773500009934000017350000C5340000BC
:10563000F53400009F360000AB3600008F330000C9
:105640009333000095360000C5320000C5320000DB
:10565000C3330000C5320000353400003F34000081
:10566000C53200009B360000C5320000B536000090
:1056700013370000113400001D340000046C0008D2
:105680000000047C03430001187801001A60400206
:10569000400C03000782000C0D0000000000000019
:1056A0003C57000005000000E40410000004000066
:1056B0000D1B0000000000000200000001000000BF
:1056C0009057000004000000E408100040060000AD
:1056D000A9220000000000000200000002000000FB
:1056E000C057000003000000240F10000008000055
:1056F0009D310000000000000200000003000000D7
:105700005C57000002000000241710000001000098
:105710003D3700000000000002000000040000000F
:105720006C570000010000002418100080000000E9
:1057300089320000000000000200000000000000AC
:105740006457000001000000010000009C570000A9
:105750000100000002000000A85700000100000046
:105760000300000078570000010000000000000066
:1057700048570000010000008457000002000000AC
:10578000B8570000030000005457000054736B5FCB
:105790005353766300000000456C665F5373766375
:1057A00000000000456C665F436D640054736B5FDE
:1057B000436D640053656D5F4166650054736B5FB4
:1057C00049646C650000000053656D5F4D5442757F
:1057D00066660000456C665F5363616E0000000002
:1057E00054736B5F5363616E0000000053656D5F1F
:1057F0004576744669666F0053656D5F43616C69F9
:10580000624672616D657300456C665F4D740000A1
:1058100054736B5F4D740000F857000000021000D5
:10582000040100001C010000FC58000000FC1000F6
:10583000040100001C010000FC58000004031000DB
:10584000401B0000380100000000000000000000C4
:105850000000000000000000000000000000000048
:105860000000000000000000000000000000000038
:105870000000000000000000000000000000000028
:105880000000000000000000000000000000000018
:105890000000000000000000000000000000000008
:1058A00000000000000000000000000000000000F8
:1058B00000000000000000000000000000000000E8
:1058C00000000000000000000000000000000000D8
:1058D00000000000000000000000000000000000C8
:1058E00000000000000000000000000000000000B8
:1058F00000000000000000000000000000000000A8
:105900000000000000000000000000000000000097
:10591000000000000000000000F00120480001200D
:105920000000000000000000000000000000000077
:105930000000000000000000000000000000000067
:1059400000000000000000000000000030B572B64A
:1059500001250D4C256000236A07012910D082F82B
:105960006B3000F03F0082F86A000848056001686B
:105970000029FCD105481C300360236062B630BDAD
:10598000402182F86B10ECE7401B00225C0D0022E6
:10599000FCB54FF00052D02082F8C3002B4F38687E
:1059A00048B140F29B70D0844520A2F85200A2F882
:1059B0005200FA2008E040F22F30D0843120A2F8C3
:1059C0005200A2F85200BC20402482F82040442516
:1059D00082F8205000234FF49676CDE900631946F3
:1059E00005E00099491E00910199491C01918142ED
:1059F000F7D30FE082F8204082F82050CDE9006311
:105A0000194605E00099491E00910199491C019130
:105A10008142F7D392F82010C906EBD482F8C33044
:105A2000386828B141F29840D08440F2572004E011
:105A300041F22C00D08440F2C110A2F85200A2F82A
:105A400052004C2082F82000FCBD0000DC04002243
:105A5000A5FA00000100004A0705194200FF961F41
:105A6000081E3240D007D00719D007000000000000
:105A700000000000000000000000070932000000E4
:105A80000000000000000000000005010A002C01D9
:105A9000C800C8000000966464005E0100009C001D
:105AA00094021405BC07C409A00F00000000000206
:105AB000000000000000000000001A0503021A04A4
:105AC00001013F02440000030001008000000000CB
:105AD0001001400660000800E50064001F0400009B
:105AE00010000001980A0B64000000000000000094
:105AF000030010051014000000000000000000006A
:105B0000020002BC02F4015802000003320A140031
:105B10000000000000000000000000000000000085
:105B2000003C000045960000050C00000301000049
:105B300006090000408000408000000000000000D6
:105B40000000000000000000000000000000000055
:105B50000000000000000000000000000000000045
:105B600000000000ECEC00EC00EC00000000000085
:105B7000000000002D3200281E1E00003C3C3C3C72
:105B80003C3C00004150003C003200000A0500147B
:105B9000000500000A0F000F0F0F0000322800322E
:105BA0003232000000000000000000000000000091
:105BB00000000000000000000000000000000000E5
:105BC00000000000000000000000000000000000D5
:105BD00000000000000000000000000000000000C5
:105BE00000000000000000000000000000000000B5
:10623000000002000000000000000000FA00000062
:106240000000000000000000000000008107073A85
:046250007E92A2098F
:00000001FF
